:100000000C94C2010C94DF010C94DF010C94DF010D
:100010000C94DF010C94DF010C94DF010C94DF01E0
:100020000C94DF010C94DF010C94BE240C949025F9
:100030000C94071F0C94DF010C94DF010C94DF017A
:100040000C94DF010C94DF010C94DF010C94DF01B0
:100050000C94DF010C948F1F0C94DF010C94DF01D2
:100060000C94DF010C94DF010C94DF010C94DF0190
:100070000C94DF010C94DF010C94DF010C94DF0180
:100080000C94DF010C94DF010C94DF010C94DF0170
:100090000C94DF010C94DF010C94DF010C94DF0160
:1000A0000C94DF010C94DF010C94DF01F405F405DE
:1000B000200620068806A606BE07BE07B1064A0728
:1000C0005B075B07FD2524261C2724261C2770269A
:1000D00093261C27EA26F926000024002500260086
:1000E0002A000000210022002300290000001E0039
:1000F0001F0020002B00F100015827003762280064
:100100000000010001000100005C0000010001008E
:1001100001005700000001000100010056002B5DA6
:100120000100010001002E0044454255473A206479
:10013000697361626C65642E0A0044454255473A12
:1001400020656E61626C65642E0A000A00253032FB
:1001500058006C65645F7461736B3A20004F6E6584
:1001600073686F743A206163746976653A20256418
:100170000A000A0025303862003A20002530325843
:10018000000A722F632030313233343536370A009B
:10019000290A002575002F002575005D28002564BB
:1001A0000020002564002000256400200025640054
:1001B0007C0025303258006D6F7573656B65792052
:1001C0005B62746E7C782079207620685D28726589
:1001D000702F61636C293A205B000A002530325889
:1001E00020006B6579626F6172645F7265706F7217
:1001F000743A20005B735D005B575D005B535D00EC
:100200005B525D005B445D005B435D001003640076
:1002100075006D006200700061006400000016034C
:1002200069006D00630068006900700077006F006E
:100230006F00640000000403090409025B0003016D
:1002400000A0FA09040000010301010009211101C5
:100250000001224000070581030800010904010094
:100260000103000000092111010001227B000705A4
:10027000820320000109040200020300000009219A
:100280001101000122220007058303200001070558
:1002900003032000011201000200000008EDFE131C
:1002A000091000010200010631FF0974A10109755E
:1002B000150026FF00952075088102097615002695
:1002C000FF00952075089102C005010902A1018572
:1002D000020901A100050919012908150025019548
:1002E00008750181020501093009311581257F95C5
:1002F000027508810609381581257F9501750881E9
:1003000006050C0A38021581257F950175088106BE
:10031000C0C005010980A101850319012AB7001594
:100320000126B700950175108100C0050C0901A1D7
:1003300001850419012AA002150126A00295017564
:10034000108100C005010906A101050719E029E790
:100350001500250195087501810295017508810137
:100360000507190029FF150026FF0095067508816D
:10037000000508190129059505750191029501757A
:10038000039101C011241FBECFEFDAE0DEBFCDBF65
:1003900011E0A0E0B1E0E8EFFFE402C005900D92AB
:1003A000A83AB107D9F722E0A8EAB1E001C01D924E
:1003B000AE38B207E1F70E9401140C94FA270C94AE
:1003C0000000FF93EF93E091A801F091A90130970D
:1003D00009F00995EF91FF910895FC018591803016
:1003E00011F0EFDFFBCF0895FF27E0E230E247FF97
:1003F0000CC0419597FF09C0EDE26095709580951E
:100400009095611D711D811D911D27FF02C02195D1
:1004100030E350E2AA27660F771F881F991FAA1F93
:10042000A41710F0A41B63955A95A9F7AA3008F0F9
:10043000A95FA05DAF93F3956115710581059105E5
:1004400041F7ED3211F4EF93F395F21718F43F935F
:10045000F395FBCF8F91B5DFFA95E1F70895E99118
:10046000F9918591803021F0853219F0AADFF9CF1A
:10047000089520E0E89455915532C1F3503311F4BA
:10048000689455915A3348F4505390F3220F022E3A
:10049000220F220F200D250FF4CF0EF42195899104
:1004A0009991533619F3533729F1533559F1BC015A
:1004B00088279927E8945C3621F48991999168946A
:1004C0005591543639F446EF7EF077FF0DC08FEF2B
:1004D0009FEF0AC055374AE039F0583540E121F026
:1004E000523642E009F00895FF93EF937DDFEF91DC
:1004F000FF91B7CFFF93EF93FC0181918030B9F367
:1005000060DFFBCFFF93EF9368DFF1CFDF93CF93F3
:10051000CDB7DEB72596A3DFCF91DF910895269A58
:10052000219A239A0C94830F2E9829982B9808953A
:10053000CF92DF92EF92FF926B017C010E94070441
:1005400080FF02C02E9A01C02E9881FF02C0299A16
:1005500001C02998C701B601FF90EF90DF90CF90BE
:100560000C94950880E090E02E9A299A2B9A2FEF10
:1005700037EE43E0215030404040E1F700C000003A
:100580002E9829982B98009749F42FEF37EE43E0E7
:10059000215030404040E1F700C000000196823019
:1005A000910511F70C94CA1280FD02C02B9A01C06C
:1005B0002B980C94690481E008950895CF93C62F79
:1005C000811118C06091BB017091BC018091BD0187
:1005D0009091BE010E940704811106C0CC2311F046
:1005E00080EF21C08FEE1FC0CC2311F08EE21BC024
:1005F0008DE219C08130C9F46091BB017091BC01DA
:100600008091BD019091BE010E940704811106C036
:10061000CC2311F089EA07C08AEA05C0CC2311F087
:100620008FE401C080E50E94A20581E0CF9108958A
:1006300081E008950C94DB0208950C941C031F9331
:10064000CF93DF9300D000D01F92CDB7DEB74983A0
:100650005A836B833091AB0189819A81311114C027
:10066000662359F0222349F00E94FB09182F682FB6
:1006700089819A810E94A20903C00E94CE09182F85
:1006800069817A81812F04C00E94FB0969817A8186
:100690000F900F900F900F900F90DF91CF911F91BF
:1006A0000C944611FC01262F408151816281738197
:1006B00084810C941F0381E00895CF93DF93EC01B4
:1006C00060E00E945203BE01DF91CF910C941D03A4
:1006D0000C94B2020C94C8120E944E080E9494021C
:1006E0002FEF84E39CE0215080409040E1F700C070
:1006F00000000C94B51F0F931F93CF93DF9300D08E
:10070000CDB7DEB78C0161E00E9452039A838983E2
:10071000B801CE0101960E948B19882309F466C0A6
:10072000B80189819A810E941A03882309F45EC066
:10073000B80189819A810E94951D882309F456C0C9
:10074000B80189819A810E941917882309F44EC043
:10075000B80189819A810E945A19882309F446C0F8
:10076000F80182818823E9F189819A818F3D2CE506
:10077000920779F140F48115FCE59F0791F08130F3
:100780009C4591F02EC08C35EDE59E0741F18D35ED
:10079000FDE59F0709F18B359D4519F50E94920EE5
:1007A00020C00E946C0322C080911F02182F109558
:1007B000117010FB80F980931F02112329F08AE346
:1007C00091E00E94ED0112C088E291E00E94ED01EB
:1007D0000EC00E94460F0AC00E94890E02C00E94ED
:1007E000950EC8010E941803182F01C010E0812F38
:1007F0000F900F90DF91CF911F910F9108950E945C
:10080000EA1E0C9478040E947B040C94F01ECF9294
:10081000DF92EF92FF926C01EE24FF24C114D10409
:10082000E104F10421F0C701B60120E101C020E09C
:10083000C72ED82EE92EFF24C114D104E104F104FF
:1008400019F0285FC701B6016B017C0154E0F694F2
:10085000E794D794C7945A95D1F7C114D104E10411
:10086000F10419F02C5FC701B6016B017C0142E075
:10087000F694E794D794C7944A95D1F7C114D1045C
:10088000E104F10419F02E5FC701B601DC01CB01D0
:10089000B695A79597958795892B8A2B8B2B09F071
:1008A0002F5F822FFF90EF90DF90CF900895829579
:1008B000982F937344E0949F900111248C7C86952B
:1008C0008695282B822F8575880F2A7A2695822B6C
:1008D0000895089581E008950C946A040895CF93D3
:1008E000C82F0E94D4028C2F0E946C04CF910895CF
:1008F00080E00C946F040E94F11D0C946F04CF9360
:100900000E94F11DC82F8091AA01C81741F1C09320
:10091000AA0180911F0282FF1EC080FF04C082E5F1
:1009200091E00E94ED0180911F0280FF0CC01F9298
:10093000CF938DE491E09F938F930E9486020F9056
:100940000F900F900F9080911F0280FF04C08BE4E6
:1009500091E00E94ED018C2FCF910C946F04CF9108
:100960000895CF93DF93CDB7DEB72B970FB6F894EA
:10097000DEBF0FBECDBF4F83588769877A878B87CD
:1009800061110E94C10D9E012F5F3F4F86E0F9016A
:1009900011928A95E9F785E0FE013796D901019019
:1009A0000D928A95E1F789819A814C815D81452B71
:1009B00031F09F3F31F491E08F3F19F403C091E093
:1009C00001C090E090FF09C049815A816B817C8110
:1009D0008D819E810E94E20C05C0C9010E945B03CB
:1009E0008111F2CF2B960FB6F894DEBF0FBECDBFAC
:1009F000DF91CF910895FC01808191810E943D0A91
:100A00000895CF93882309F450C0C82F8CEF8C0F22
:100A1000813AD0F46C2F80910201909103010E94E1
:100A20008C1E882349F06C2F809102019091030164
:100A30000E94C41E0E94E30D6C2F809102019091D0
:100A400003010E94C21E0CC080E28C0F883058F453
:100A5000C77081E001C0880FCA95EAF70E94A40D13
:100A6000CF910C94E30DEBE5EC0FE33040F4F0E0B4
:100A7000E95BFE4F808190E0CF910C94541EE8E535
:100A8000EC0FE73150F4F0E0EE0FFF1FE75EFE4F92
:100A900080819181CF910C946A1ECD3E30F08C2FD5
:100AA0000E948614CF910C945815CF9108958823F5
:100AB00089F19CEF980F913A40F4682F80910201E0
:100AC000909103010E94C41E0DC090E2980F9830CF
:100AD00058F4877091E001C0990F8A95EAF7892F41
:100AE0000E94AA0D0C94E30D9BE5980F933020F41F
:100AF00080E090E00C94541E98E5980F973120F414
:100B000080E090E00C946A1E8D3E20F00E94E1147B
:100B10000C94581508951F93CF93DF93182FEB0172
:100B20000E940105209741F08FE99FE00197F1F7BE
:100B300000C000002197F6CF812FDF91CF911F9148
:100B40000C945705893319F060E070E002C060E54D
:100B500070E00C948B05882321F00E94A40D0C9466
:100B6000E30D0895882321F00E94AA0D0C94E30D53
:100B70000895CF92DF92EF92FF920F931F93CF933E
:100B8000DF937C01D62FC72FFC01128105810295CE
:100B90000F700E949A0D8823B9F01123A9F08C2FB1
:100BA000807F803421F080E28D0F883068F0809162
:100BB000740282FD09C082E00E94430E0E949A0DD9
:100BC00091E0D82ED92601C0D12CCC2EC2948FE032
:100BD000C8228C2D90E08C30910508F0CFC1FC012B
:100BE000EA5AFF4F0C946F278C2F807FCF70882399
:100BF00011F0C295C07F112399F0CC2309F4AAC14A
:100C000080E28D0F883010F0D11104C08C2F0E942B
:100C1000A40D03C08C2F0E94B40D0E94E30D9AC155
:100C20008D2F0E945705CC2309F4A8C180E28D0FB7
:100C3000883038F1DD2329F18C2F0E94BA0D24C0B1
:100C40008C2F807FCF70803211F0C295C07FDD2362
:100C500019F0D130A1F13DC08091740282FF17C01C
:100C6000112349F0CC2329F08C2F0E94A40D0E945F
:100C7000E30D80E070C180E00E945705CC2309F4A9
:100C80007DC18C2F0E94AA0D0E94E30D77C1112314
:100C900071F0002341F0013031F40E94C40D8C2B1F
:100CA0000E94CC0D6BC10E94C40D8C2B1DC0002373
:100CB00019F0013009F462C10E94D90D25C0112339
:100CC00021F0033008F05AC10EC0023008F056C1BE
:100CD0001BC0112361F0002331F0F701858180FFF3
:100CE00039C18F7085838C2F0E94AB0547C10023CB
:100CF00059F0D93309F03FC1FFEF07EE13E0F1508F
:100D000000401040E1F735C18C2F0E94B20536C17A
:100D10008C2F86958695837019F0813061F02EC1F5
:100D2000112321F08D2F9C2F937002C080E090E062
:100D30000E94541E2BC1112321F08D2F9C2F9370E4
:100D400002C080E090E00E946A1E20C18D2F112316
:100D500019F00E94861402C00E94E1140E945815E6
:100D600015C18C2F837009F047C011110BC12D2FB5
:100D7000229526952770220F220F6D2F6F70862FD8
:100D800090E0A0E0B0E0022E04C0880F991FAA1FD7
:100D9000BB1F0A94D2F7D4FF10C04FE050E060E0D0
:100DA00070E004C0440F551F661F771F2A95D2F7C5
:100DB000409550956095709503C040E050E0BA01B1
:100DC000C695C695C3708A019B01082B192B2A2B47
:100DD0003B2BC901B801C23049F058F4C13019F0B9
:100DE0000E94BA08CFC00E94A808CCC00E94CC08BC
:100DF000C9C00E94A608C6C0112319F08C2F8170AB
:100E000001C08695882309F4BDC02D2F2295269513
:100E10002770220F220F6D2F6F70862F90E0A0E0B9
:100E2000B0E0022E04C0880F991FAA1FBB1F0A94AE
:100E3000D2F7D4FF10C04FE050E060E070E004C093
:100E4000440F551F661F771F2A95D2F7409550957E
:100E50006095709503C040E050E0BA01C695C69514
:100E6000C3708A019B01082B192B2A2B3B2BC9012C
:100E7000B801C23049F058F4C13019F00E947D0920
:100E800081C00E946B097EC00E948F097BC00E94B6
:100E9000DE0878C0CF70112339F08C2F0E9404092E
:100EA0008D2F0E94AB056EC08D2F0E94B2058C2F36
:100EB0000E94250967C0D23F21F128F4D03F41F0BC
:100EC000D13FC1F043C0D33F19F1D43F79F03EC0C8
:100ED000112341F0023008F051C08C2F8F710E9415
:100EE0004A094CC0033008F049C0F7CF8091740222
:100EF00082FF18C0112339F08C2F8F710E940409D2
:100F00003DC01123C9F38C2F8F710E94250936C073
:100F1000112329F08C2F8F710E94EF082FC00E949F
:100F2000EA082CC0112349F0CF718C2F0E940409CC
:100F300063E08C2F0E94280E21C081E00E94430EA6
:100F40000230E0F082E00E94430E18C0112331F01D
:100F5000002391F28D2F0E94010510C0002399F209
:100F6000D93349F41FEF27EE33E0115020403040D1
:100F7000E1F700C000008D2F0E94570588EF8C0D0F
:100F8000843020F40E94F11D0E946F04DD20C9F01E
:100F90000E94960D80FD15C0F70112820E94900DEF
:100FA0000E940409C7010E9402080E94900DDF916F
:100FB000CF911F910F91FF90EF90DF90CF900C9405
:100FC0002509DF91CF911F910F91FF90EF90DF9056
:100FD000CF9008950F931F93CF93DF93EC01688117
:100FE00079818A810E94480A8C010E94A1090E948D
:100FF0009408B801CE010E94B905DF91CF911F91ED
:101000000F910895CF93DF93EC01988189812B8113
:101010003C81232B31F08F3F31F481E09F3F19F465
:1010200003C081E001C080E080FD1DC0CE010E94B0
:101030007B03811110C00E949A0D8823A1F08A8140
:10104000882389F08091740282FD0DC082E0DF91D7
:10105000CF910C94430ECE010E94EA07CE01DF919E
:10106000CF910C945D03DF91CF91089580E090E0E3
:101070000E94541E80E090E00E946A1E0E94C10DF2
:101080000E94E30D0E940B170C94581580910201E9
:10109000909103010E94C61E0C9436080E94B10D67
:1010A0000C94460892959F70963079F010F4925007
:1010B00001C09A50923068F4803F69F018F4883E7D
:1010C00040F409C0843F29F406C0883E20F0813FE7
:1010D00011F080E0089581E00895FC018081918104
:1010E0000E943D0A0E9452080895CF93DF9300D0DA
:1010F00000D01F92CDB7DEB70F900F900F900F90DA
:101100000F90DF91CF910895CF93DF9300D000D05F
:1011100000D0CDB7DEB726960FB6F894DEBF0FBE6F
:10112000CDBFDF91CF910895089508950C9495084F
:101130000C9496080E9498086093BF017093C001B8
:101140008093C1019093C2010C9436080C949A08C4
:101150000F931F930091BF011091C0012091C10115
:101160003091C201602B712B822B932B1F910F9119
:101170000C949A080F931F930091BF011091C00126
:101180002091C1013091C2016023712382239323F6
:101190001F910F910C949A080F931F930091BF0118
:1011A0001091C0012091C1013091C20160277127C7
:1011B000822793271F910F910C949A080E949802FE
:1011C0006093BB017093BC018093BD019093BE01FD
:1011D0000C94360860E070E0CB010C94DE080F93AD
:1011E0001F9341E050E060E070E08A019B0104C081
:1011F000000F111F221F331F8A95D2F7C901B801B2
:101200001F910F910C94DE080F931F9341E050E063
:1012100060E070E004C0440F551F661F771F8A9579
:10122000D2F78091BB019091BC01A091BD01B0911A
:10123000BE018A019B01082B192B2A2B3B2BC901CC
:10124000B8011F910F910C94DE080F931F9341E09A
:1012500050E060E070E004C0440F551F661F771F28
:101260008A95D2F740955095609570958091BB0115
:101270009091BC01A091BD01B091BE018A019B017A
:10128000082319232A233B23C901B8011F910F9179
:101290000C94DE080F931F9341E050E060E070E093
:1012A00004C0440F551F661F771F8A95D2F780919F
:1012B000BB019091BC01A091BD01B091BE018A011A
:1012C0009B01082719272A273B27C901B8011F912D
:1012D0000F910C94DE080F931F930091BB011091A6
:1012E000BC012091BD013091BE01602B712B822B7E
:1012F000932B1F910F910C94DE080F931F93009175
:10130000BB011091BC012091BD013091BE01602351
:101310007123822393231F910F910C94DE080F9366
:101320001F930091BB011091BC012091BD01309130
:10133000BE0160277127822793271F910F910C947C
:10134000DE08089524E0929F900D1124890FE82F64
:10135000E695E695E695877051E001C0550F8A95B0
:10136000EAF785E0E89FF0011124E455FE4F20E004
:1013700030E070E04081CB01022E02C09695879547
:101380000A94E2F7817081958427852384278193CD
:101390002F5F3F4F2530310569F7089524E0929F74
:1013A000900D1124890F682F669566956695982F84
:1013B000977085E0689FB001112440E050E080E024
:1013C000FB01E40FF51FE455FE4F208130E0092EAC
:1013D00002C0369527950A94E2F721703327042E30
:1013E00001C0220F0A94EAF7822B4F5F5F4F45300E
:1013F000510531F70895BF92CF92DF92EF92FF929D
:101400000F931F93CF93DF938C01C090BB01D090BB
:10141000BC01E090BD01F090BE018091BF019091B0
:10142000C001A091C101B091C201C82AD92AEA2AFB
:10143000FB2ACFE1D0E0D701C6010C2E04C0B6953F
:10144000A795979587950A94D2F780FD04C02197B8
:1014500090F7B12C07C0BC2EB8018C2F0E945911F7
:101460000197A9F38B2DDF91CF911F910F91FF90E1
:10147000EF90DF90CF90BF900895CF93DF93EC0172
:101480000E94FB09BE010E945911DF91CF9108957E
:101490001F93CF93DF93EB019091AB01992321F040
:1014A000CB010E943D0A13C0882349F0CB010E9462
:1014B000FB09182F682FCE010E94A20904C0CB019E
:1014C0000E94CE09182FBE01812F0E945911DF9171
:1014D000CF911F9108951F93CF93DF93C091C301C4
:1014E00016E08091C401C81799F0D0E01C9FF0016C
:1014F0001D9FF00D1124EB53FE4F408151816281FD
:101500007381848195810E9484082196C770E9CFF8
:10151000DF91CF911F9108954091F5015091F6010F
:101520006091F7017091F8018091F9019091FA01B1
:101530000C948408EF92FF920F931F93CF93DF9345
:101540008091FA0182958F7009F065C08091F70152
:10155000882309F460C08091C301F090C401109108
:10156000F5010091F6016091F8017091F90191E0A7
:101570001F3F09F090E0C0910001D0910101292F97
:1015800096E0E92E8F1509F446C06115710521F02A
:101590000F3F21F030E003C031E001C0322F90E076
:1015A00030FD36C0E89EF001E99EF00D1124DF0108
:1015B000AB53BE4F11963C911197301329C03C910B
:1015C000311326C012963C911297311121C0139607
:1015D0004D915C911497461B570B4C175D07C0F457
:1015E0008091FA018F7080618093FA01E653FE4F7B
:1015F00080818F708061808385EF91E00E94020876
:10160000DF91CF911F910F91FF90EF900C946B0A97
:1016100001968770B7CFDF91CF911F910F91FF9007
:10162000EF9008959F92AF92BF92CF92DF92EF9288
:10163000FF920F931F93CF93DF93CDB7DEB76197E0
:101640000FB6F894DEBF0FBECDBF8C0185E0F80168
:10165000DE011D9601900D928A95E1F7D801129650
:10166000EC909091F501E091F6012091F801309114
:10167000F9012115310531F0EF3F31F481E09F3F51
:1016800019F403C081E001C080E0B82FB1709B2E37
:1016900080FD47C1D8014C9111965C91119713962A
:1016A000AD90BC90149785EFC82E81E0D82EF090B5
:1016B000F701B501621B730B20910001309101010C
:1016C000FF2009F4D9C08091FA016217730708F06E
:1016D00095C0282F207F09F052C05E1313C0491314
:1016E00011C0FE2CE1100EC08F7080618093FA0152
:1016F0000E948C0AC6010E9402088091FA01F8013A
:1017000085834DC1AB2831F05F3F31F481E04F3F1D
:1017100019F403C081E001C080E080FD03C081E0D6
:101720008E2502C080E090E0F82FF170FF2E80FF40
:101730001CC08091C3012091C40136E0821709F4D6
:101740000BC190E0389FF001399FF00D1124EB534D
:10175000FE4F6181561306C06081461303C062814B
:10176000E61203C001968770E9CFFE2CEE2009F443
:1017700016C18091FA0181608093FA0154C05E1312
:1017800006C0491304C0E11002C0F80199C0C801A5
:101790000E946D08882361F1EE2051F12091FA0139
:1017A000822F82958F7090E0029774F08091F501FE
:1017B0009091F60198878F831986BB86AA862C871D
:1017C000CE0107960E94020886E0F801A5EFB1E07D
:1017D00001900D928A95E1F70E949A0A0E948C0A64
:1017E0000AC05E1711F1C8010E946D0881112CC05A
:1017F000C8010E940208FF24F394D1C0282F207F43
:1018000081F77A2DB98AA88A6E2D89890E94750878
:1018100085EF91E00E94020886E0D6011D928A952C
:10182000E9F70E948C0AF12CBAC04913DCCFE11011
:10183000DACFF8018583C8010E94020886E0D6014C
:101840001D928A95E9F7ABC0EE2091F22091FA0142
:10185000822F82958F7090E002970CF4B5CF809123
:10186000F5019091F6019A8389831B82BD82AC8237
:101870002E83CE010196A6CF6217730708F044C0ED
:10188000FE2CEE2009F4B4CF5E1330C049132EC0F5
:101890002091FA0120FD21C0822F82958F70482F60
:1018A00050E041155105C9F0F80125834F3051052D
:1018B00041F08F5F982F9295907F822F8F70892BA8
:1018C0008583C8010E94020886E0F801A5EFB1E017
:1018D00001900D928A95E1F73CC086E0F801A5EFF2
:1018E000B1E001900D928A95E1F759C0C8010E94BC
:1018F0006D08811169CF8091FA0181608093FA01AE
:10190000C8010E9402084BC07A2DB98AA88A6E2DA0
:1019100089890E94750886E0D6011D928A95E9F7AB
:1019200018C0EE2009F464CFC8010E946D08F82E9B
:10193000882309F45DCF86E0F801A5EFB1E00190BE
:101940000D928A95E1F785EF91E00E94FB040E94D9
:101950009A0A0E948C0A23C04D875E878D859E85DA
:101960000E943D0A292F22952F70223028F49F7063
:1019700039F0811105C00BC0243028F49F7049F460
:10198000805E883020F0C8010E9402089F2CF92C4C
:1019900006C0D80115969C91907F91F7F8CF8F2DB6
:1019A00061960FB6F894DEBF0FBECDBFDF91CF9129
:1019B0001F910F91FF90EF90DF90CF90BF90AF906D
:1019C0009F9008951F93CF93DF93CDB7DEB72C97E9
:1019D0000FB6F894DEBF0FBECDBF4F83588769871F
:1019E0007A878B879C87CE0107960E94120B8823EB
:1019F000D1F09F8188852A853B85232B31F08F3F4D
:101A000031F481E09F3F19F403C081E001C080E020
:101A100080FD47C04F81588569857A858B859C8577
:101A20000E9484083EC086E0FE013796DE011196D2
:101A300001900D928A95E1F7FF81E8856A857B85A3
:101A40006115710531F0EF3F31F481E0FF3F19F48A
:101A500003C081E001C080E080FD23C02091C4016B
:101A600030E0C9010196877099274091C30150E089
:101A700084179507F1F1F983EA837D836C8396E0FF
:101A8000929FD001939FB00D1124AB53BE4FFE0126
:101A9000319601900D929A95E1F78093C4010E94CE
:101AA0006B0A16E08091C3019091C401891771F10E
:101AB000189FC00111248B539E4F0E94120B882344
:101AC00029F1E091C3011E9FF0011124EB53FE4F59
:101AD0004081518162817381848195810E94840853
:101AE0008091C30190E00196877099278093C3018C
:101AF000D9CF0E944E081092C4011092C301E5EFA5
:101B0000F1E086E0DF011D928A95E9F72C960FB689
:101B1000F894DEBF0FBECDBFDF91CF911F91089526
:101B2000809103028595859585950895809103029E
:101B30008770089590910302977081E009F480E026
:101B4000089580910E02089590910E02892B809342
:101B50000E020895809590910E02892380930E02C3
:101B6000089510920E02089590910D02892B809392
:101B70000D020895809590910D02892380930D02A6
:101B8000089510920D020895809104020895089519
:101B90000C94C70D0C94C80D9091740292FD08C06E
:101BA00090910402981721F0809304020C94CA0DBE
:101BB000089580910402882329F01092040280E0A5
:101BC0000C94CA0D0895CF93DF93E0910201F09138
:101BD000030180910E028083E0910201F0910301E4
:101BE000908180910D02892B80838091040288234B
:101BF00081F0E0910201F09103019081892B8083B3
:101C000080910201909103010E94801E81110E9427
:101C1000D90DC0910201D091030148E050E06BEF73
:101C200071E0CE010E94AB27892B69F088E0FE01AC
:101C3000ABEFB1E001900D928A95E1F7CE01DF9113
:101C4000CF910C94FD1DDF91CF9108950C94C70D99
:101C50009091740292FD10C098E0899F9001112428
:101C6000262B209303020E9404098091030285958C
:101C7000859585950C94260E0C9404091092030208
:101C800080E00C94260E209103028095822380939D
:101C90000302982F977099F430E0482F082E000C1B
:101CA000550B2417350759F09091740292FD07C027
:101CB0008595859585950E9425090C943E0E08957D
:101CC000CF939091740292FB222720F92817F9F004
:101CD000C82F892FC0FB82F9809374028091730210
:101CE000909174020E94C20E82E00E94430E809185
:101CF0001F0280FF0CC01F92CF938DE591E09F9350
:101D00008F930E9486020F900F900F900F90CF91AB
:101D100008958091740282FB882780F991E08927D9
:101D20000C94600E81E00C94600E80E00C94600EC8
:101D30006FEF7FEF80E090E00C94E42780E090E08C
:101D40000E94C02721E0893E9E4F09F020E0822FAB
:101D5000089582E090E00C94B82783E090E00C9422
:101D6000B827CF9384E090E00E94B827C82F82E282
:101D700090E00E94B8272C2F30E0A901582BCA010F
:101D8000CF910895CF93C92F682F84E090E00E94EF
:101D9000C6276C2F82E290E0CF910C94C627AB014E
:101DA000BC018FE090E00C94D827AB01BC0183E12B
:101DB00090E00C94D82760E070E0CB010C94D50E35
:101DC00060E070E0CB010E94CF0E0C94DB0E69EE58
:101DD0007EEF80E090E00E94E42760E082E090E007
:101DE0000E94C62760E083E090E00E94C627109220
:101DF000BF011092C0011092C1011092C20160E0B7
:101E000084E090E00E94C62760E082E290E00E94B9
:101E1000C62760E085E090E00E94C62760E086E08B
:101E200090E00E94C6276FEF87E090E00E94C627EF
:101E300040E050E0BA0188E090E00E94D82760E0DE
:101E40008DE090E00E94C62740E050E0BA0188E1B2
:101E500090E00E94D82760E087E190E00E94C627CA
:101E600040E050E0BA018CE190E00E94D82760E0A9
:101E700070E080E290E00E94E42740E050E0BA0188
:101E800088E190E00E94D8270C94E00E0C94E70EB5
:101E9000682F8EE090E00C94C6270E94741F609318
:101EA0001B0270931C0280931D0290931E0260938C
:101EB0001702709318028093190290931A020895E2
:101EC0000E94741F60931B0270931C0280931D027A
:101ED00090931E0260931302709314028093150274
:101EE00090931602089585B7806885BF85B780688E
:101EF00085BF089581E008950C947A0F08950C949D
:101F00007E0F0C94DD020C947E0F0C947E0F0E94C9
:101F1000730F89E991E20E94E71D0E94850F0C94DE
:101F20008F020E947F0F0C947E0F0E944D120C9422
:101F30006E040E945F1F0E9467130E94950F0E940B
:101F40006A180C94810F8F929F92AF92BF92CF929A
:101F5000DF92EF92FF920F931F93CF93DF93CDB752
:101F6000DEB72A970FB6F894DEBF0FBECDBF0E9432
:101F70007C13982E81110E944D0F8FE0A82E82E0D5
:101F8000B82E00E010E0802E802F0E947112D82E13
:101F9000F501C1905F01C826B1F40F5F1F4F0430F7
:101FA000110589F78FEF89838A831B820E94681F3E
:101FB0008160782F9D838C8349815A816B818D81CB
:101FC0000E94B1042FC080911F0281FD0E947712F0
:101FD000E12CFF24F3948C2D8F21F1F00E947C0FD3
:101FE000882399F0EE828F82DF2081E009F480E07F
:101FF00088870E94681F8160782F9A8789874E8121
:102000005F8168858A850E94B104F801E15FFD4F18
:102010008081F826F08206C0E394FF0CF5E0EF1211
:10202000DACFBBCF81E0911001C080E02A960FB6D5
:10203000F894DEBF0FBECDBFDF91CF911F910F91FE
:10204000FF90EF90DF90CF90BF90AF909F908F90D8
:1020500008950E94A30F0E94BD1881110E94600F75
:102060000E94F8150C947F04CF93DF930E945E11B9
:10207000EC01811521E5920708F045C0811530E596
:10208000930708F094C0883E910528F5803E91059D
:1020900008F0F8C0883A910570F4853A910508F087
:1020A0007CC08130910509F475C008F4E8C004973C
:1020B00008F0E8C0E4C08F3B910508F0E0C0C85AC2
:1020C000D0E0CC0FDD1FC65BDE4F0990D881C02D5C
:1020D000CE019464D8C0811540E2940758F481156C
:1020E00051E0950708F0CEC08D3E910508F4C7C0B9
:1020F0009065C9C0C11580E4D80708F4C0C0DF707E
:10210000CE01906AC0C0811525E59207A8F481151B
:1021100034E5930708F095C0811543E5940708F06E
:102120007BC0811552E5950708F061C0D82FCC27F8
:10213000CE01816F906AA7C0C11589E5D807A0F4C8
:10214000C11528E5D20708F082C0C11536E5D307CE
:1021500008F095C08C2F0E94F2118F7190E0D82F5B
:10216000CC27CE0190628FC0C1154AE5D40708F490
:1021700074C0CE0190568115904208F080C08D2F1A
:102180008F710E94F211DD27D0628F71AE01582B42
:10219000CA0179C081E090E076C0C55AD0E0C85845
:1021A000DE4F8881C82FD0E0CE0190646CC074E00F
:1021B000969587957A95E1F7282F23703C2F3370F9
:1021C00081E090E002C0880F991F3A95E2F79C6881
:1021D000AC01522B9A019C2F9F709695969550E2D8
:1021E000959FE0011124C9018C2B9D2B4CC083705D
:1021F000992721E030E002C0220F331F8A95E2F7D1
:102200009C2F9695969580E2989FE0011124C22B11
:10221000D32BCE019C6837C08370992721E030E032
:1022200002C0220F331F8A95E2F79C2F9695969550
:1022300040E2949FE0011124C22BD32BCE019A6877
:1022400022C0D82FCC27CE01846F906A1CC0DC2F0F
:10225000CC27CE01806F906A16C08C2F8F700E94A1
:10226000F21194E0D695C7959A95E1F7CF70D0E03A
:10227000DC2FCC27D0699E01282BC90104C080E047
:1022800090E001C0CE01DF91CF91089524E1829FBB
:10229000C0011124FC0125E0729FE00DF11D112405
:1022A000E60FF11DEE0FFF1FE852FF4F859194914D
:1022B00008950E9446110E943410089582389105B5
:1022C00069F1B0F48133910509F46DC048F48932A5
:1022D000910509F463C08A32910509F469C0089533
:1022E0008533910509F455C089339105B9F00895F6
:1022F000833E910569F138F4803E9105B1F0823E4C
:10230000910509F10895863E9105A9F1873E910551
:10231000B9F1843E910509F064C023C02091730295
:1023200020FD4FC021FD4DC008958091730280FDB6
:1023300044C08091740280FF44C08091730284FD88
:1023400042C083EE4DC08091730282FF38C0F5CF4A
:102350008091730282FD33C08091740280FD31C090
:10236000ECCF8091740281FF32C08091730284FDB2
:102370002AC087EE35C08091730283FF26C0F5CF57
:102380008091730283FD21C08091740281FD1FC082
:10239000ECCF8091730285FD1CC01DC0809173023B
:1023A00085FD19C016C08091730286FD16C017C046
:1023B0008091730286FD13C010C089E311C082EEC4
:1023C0000FC080EE0DC080E00BC086EE09C084EE29
:1023D00007C089E205C085E303C08AE201C081E34A
:1023E00090E008959091730292FF0DC0282F2871FC
:1023F000283019F4877F846006C0282F2471243088
:1024000011F48B7F886093FF0DC0282F287128312D
:1024100019F4877E846106C0282F2471243111F4B9
:102420008B7E88612091740220FF0DC0382F387197
:10243000383019F4877F816006C0382F3171313010
:1024400011F48E7F886021FF0DC0282F287128315C
:1024500019F4877E816106C0282F2171213111F482
:102460008E7E886194FD877E08950C94980E0E945C
:102470007C138FE39CE90197F1F700C000000E94F4
:102480007C1383E00E94711280FF04C00E94351209
:102490000C94B51F08950C9437120E949E0E811162
:1024A00002C00E94460F0E94A90E80931F020E9444
:1024B000B10E90937402809373020E944B120E949B
:1024C000AD0E682F70E080E090E00E94A608609159
:1024D000BB017091BC018091BD019091BE010C9433
:1024E0009802E82FF0E0E758FD4F80810895CF92E1
:1024F000DF92EF92FF920F931F93CF93DF9381E8C8
:1025000091E00E94ED0189E7E82E82E0F82EC0E01C
:10251000D0E09CE7C92E91E0D92E04E711E0DF93CB
:10252000CF93DF92CF920E94860289E791E00E94CA
:10253000ED01F70181917F010E9457041F928F9353
:102540001F930F930E94860282E791E00E94ED01A3
:1025500021968DB79EB708960FB6F8949EBF0FBE12
:102560008DBFC430D105D9F6DF91CF911F910F9166
:10257000FF90EF90DF90CF90089580EA8A95F1F771
:10258000089500C008950C94BD1208950C94C512CE
:102590000C94C6120C94C512F894E82FE295EF70D3
:1025A000F0E031A1282F2F7081E090E001C0880F6A
:1025B0002A95EAF7982F9095932391A392A1892BBE
:1025C00082A3789408950F931F93CF93DF93C0E86D
:1025D000D1E089918F3F11F00E94CC1281E0C43884
:1025E000D807B9F7CBE7D1E000E811E089918F3F38
:1025F00011F00E94CC120C171D07C1F7DF91CF918B
:102600001F910F910895CF92DF92EF92FF920F9357
:102610001F93CF93DF938C01C62FD0E0CE0180585B
:102620009E4F7C01FC0190819F3F09F447C0D62E4C
:10263000F894E92FE295EF70F0E081A19F7021E01E
:1026400030E001C0220F9A95EAF7822B81A382A184
:102650002095282322A378940E94C112EBE7F1E091
:1026600040E851E031E0C12C21912F3F89F0A22FA9
:10267000A295AF70B0E090968C9190E02F7002C060
:10268000959587952A95E2F780FD02C0832F01C0BA
:1026900080E0C82A330F4E175F0731F7F7018081BA
:1026A0008F3F11F00E94CC1261E0C11001C060E0C8
:1026B0008D2D0E94C312C00FD11FC882DF91CF9110
:1026C0001F910F91FF90EF90DF90CF9008950E949F
:1026D000E31284E0E9E7F2E0DF01982F1D929A957A
:1026E000E9F7E5E7F2E0DF011D928A95E9F784E07A
:1026F0000E94BE130C9468031F93CF93DF9300D006
:1027000000D0CDB7DEB719821A821B821C8210E07E
:10271000612FCE0101960E9403131F5F1430C1F791
:1027200044E050E0BE016F5F7F4F85E792E00E947A
:10273000AB2711E0009709F410E0892B61F0898143
:102740009A81AB81BC818093750290937602A093AD
:102750007702B0937802212F44E069E772E085E7C1
:1027600092E00E94BF130E946A03812F0F900F9086
:102770000F900F90DF91CF911F9108950895FF92D0
:102780000F931F93CF93DF938C01F62ED72FC42F77
:10279000222349F081E0809322020E94681F9093D7
:1027A000210280932002809122028823C1F080912F
:1027B0002002909121020E94801F059780F0EF2D4A
:1027C000FD2FD8014C2F50E0CD01801B910B8417B9
:1027D00095071CF48D918193F7CF10922202DF911F
:1027E000CF911F910F91FF9008950E9415220E9492
:1027F000990F0C9421220E9425220E9429100C94EA
:1028000043220E94061F0E94FC210E94870F0E9403
:10281000F5130E94FB130E94910FFBCF80912902B8
:1028200080FF06C06091090170E0660F771F26C027
:1028300081FF04C06091090184E005C082FF07C0E8
:102840006091090188E0689FB001112417C0909140
:1028500028029923D1F060910801961788F72091FA
:10286000090188E0289F90011124929FA001939F65
:10287000500D112470E0CA010E945B276038710579
:1028800040F46115710519F406C068E070E0862F08
:1028900008958FE7089581E008958091290280FFCF
:1028A00008C06091050170E075956795759567950D
:1028B00021C081FF06C06091050170E075956795A4
:1028C00019C082FF04C06091050170E010C09091B2
:1028D0002702992399F0609104019617A0F780913F
:1028E0000501899FC001112470E00E945B276038B8
:1028F000710540F46115710519F406C061E070E0DE
:10290000862F08958FE7089581E008958D3E21F484
:102910000E940E14819504C08E3E29F40E940E146C
:1029200080932D0208958F3E21F40E940E1481950C
:1029300004C0803F29F40E940E1480932C02089555
:10294000893F19F40E944D1405C08A3F31F40E945A
:102950004D14819580932E0208958B3F21F40E949F
:102960004D14819504C08C3F29F40E944D1480932E
:102970002F0208959FE0980F983078F421E030E01E
:10298000A90102C0440F551F9A95E2F7CA01909120
:102990002B02892B80932B0208958D3F21F4809187
:1029A000290281600BC08E3F21F480912902826050
:1029B00005C08F3F29F48091290284608093290209
:1029C00008958D3E39F490912D0297FF35C01092F5
:1029D0002D0259C08E3E29F490912D021916BCF398
:1029E0002BC090912C028F3E29F497FF25C01092A6
:1029F0002C0249C0803F19F41916CCF31DC09091E8
:102A00002E02893F29F41916BCF410922E023BC005
:102A10008A3F19F497FF10C0F8CF8B3F39F490919B
:102A20002F0297FF09C010922F022DC08C3F21F476
:102A300090912F021916BCF39FE0980F983080F404
:102A400021E030E0A90102C0440F551F9A95E2F73A
:102A5000CA01809590912B02892380932B0213C089
:102A60008D3F21F4809129028E7F0BC08E3F21F48F
:102A7000809129028D7F05C08F3F29F48091290222
:102A80008B7F8093290280912C02811106C0809156
:102A90002D02811102C01092280280912E02811114
:102AA00006C080912F02811102C010922702089562
:102AB00080911F0283FF7EC087EB91E00E94ED01B1
:102AC00080912B021F928F9382EB91E09F938F93C3
:102AD0000E94860280EB91E00E94ED0180912C0221
:102AE000282F082E000C330B3F938F938DEA91E033
:102AF0009F938F930E9486028BEA91E00E94ED01E2
:102B000080912D02282F082E000C330B3F938F93BA
:102B100088EA91E09F938F930E94860286EA91E073
:102B20000E94ED0180912E02282F082E000C330BFD
:102B30003F938F9383EA91E09F938F930E94860245
:102B400081EA91E00E94ED0180912F02282F082E4A
:102B5000000C330B3F938F938EE991E09F938F93FB
:102B60000E9486028BE991E00E94ED01809128028B
:102B70001F928F9388E991E09F938F930E94860222
:102B800086E991E00E94ED01809129021F928F93C6
:102B900083E991E09F938F930E94860280E991E000
:102BA0000E94ED018DB79EB74C960FB6F8949EBF6C
:102BB0000FBE8DBF0E94681F20912C02211104C0FE
:102BC00020912D02222321F090932602809325024A
:102BD00020912E02211104C020912F02222321F0E6
:102BE00090932402809323028AE292E00C94461E82
:102BF000EF92FF920F931F93CF93DF9300D000D0FB
:102C000000D0CDB7DEB786E0EAE2F2E0DE01119651
:102C100001900D928A95E1F7E0902C02F0902D0240
:102C200000912E0210912F0210922C0210922D0270
:102C300010922E0210922F02E11003C0FF2009F41F
:102C40005DC080912502909126020E94801FAC01F8
:102C500090912802992339F020910A0130E024173D
:102C6000350758F04BC020910B018AE0289F900156
:102C700011242417350718F041C09F3F19F09F5FBA
:102C800090932802EE2061F00E940E141E1414F09E
:102C90009FEF01C091E0989F902D112490932C02FA
:102CA000FF2061F00E940E141F1414F09FEF01C06A
:102CB00091E0989F902D112490932D0230912C0239
:102CC0003323E1F020912D022223C1F045EB3403A0
:102CD000C0011124992319F090932C0203C081E0C4
:102CE00080932C0235EB2303C0011124992319F0A2
:102CF00090932D0203C081E080932D02011103C047
:102D0000112309F45DC080912302909124020E9456
:102D1000801FAC0190912702992339F02091060180
:102D200030E02417350758F04BC0209107018AE0A6
:102D3000289F900111242417350718F041C09F3FA8
:102D400019F09F5F90932702002361F00E944D14B9
:102D5000101614F09FEF01C091E0989F902D112460
:102D600090932E02112361F00E944D14111614F05D
:102D70009FEF01C091E0989F902D112490932F0216
:102D800030912E023323E1F020912F022223C1F053
:102D900045EB3403C0011124992319F090932E02BE
:102DA00003C081E080932E0235EB2303C001112480
:102DB000992319F090932F0203C081E080932F0292
:102DC00080912C0281110BC080912D02811107C0CE
:102DD00080912E02811103C080912F0281110E94E7
:102DE0005815EB82FC820D831E8386E0FE0131962E
:102DF000AAE2B2E001900D928A95E1F726960FB60D
:102E0000F894DEBF0FBECDBFDF91CF911F910F9120
:102E1000FF90EF900895EAE2F2E086E0DF011D9274
:102E20008A95E9F71092280210922702109229023F
:102E30000895CF93DF93EC01FB018281882309F48D
:102E40003CC1C430FDE5DF0760F4CB3F9CE5D9070A
:102E500088F49E0122503C452431310508F02EC1F2
:102E600009C0C236EDE5DE0729F0C63AFDE5DF0709
:102E700009F024C10E94B10E9093740280937302F2
:102E8000C1318CE5D80709F4C6C008F042C0C9308A
:102E9000ECE5DE0709F49BC000F5C5308CE5D807EA
:102EA00009F485C078F4C330ECE5DE0709F478C096
:102EB00008F07AC0C230DC4509F0F5C08091730299
:102EC0008160EFC0C7309CE5D90709F478C008F0ED
:102ED0007AC0809173028061E4C0CD30FCE5DF07E9
:102EE00009F487C058F4CB309CE5D90709F479C0C0
:102EF00008F07BC08091730288606FC0CF30FCE522
:102F0000DF0709F480C008F082C080917302877FD8
:102F1000C8C0CE3F9CE5D90709F471C000F5C531A2
:102F2000FCE5DF0709F485C068F4C3319CE5D907E7
:102F300009F475C008F095C00E944E088091730294
:102F40008F77AFC0CC3FFCE5DF07A9F108F054C094
:102F5000CB3FDC4509F0A7C08091740240C0C2306D
:102F6000EDE5DE0709F489C058F4C1158DE5D807F1
:102F700009F45AC008F069C08091740282602FC0C1
:102F8000C236EDE5DE0709F47CC0C63AFDE5DF0791
:102F900009F481C0C330DD4509F085C080E06EC012
:102FA0008091730282607DC08091730216C080910F
:102FB0007302886076C08091740282604FC08091F5
:102FC000730280626EC08091730280646AC00E9446
:102FD0004E0880917302806864C0846062C0816022
:102FE0003DC0809173028E7F5CC0809173028D7FA3
:102FF00058C08091730216C08091740218C08091ED
:1030000074028D7F2BC0809173028F7E4AC08091A5
:1030100073028F7D46C0809173028F7B42C0809186
:103020007302877F8B7F3DC0809174028D7F8E7F7E
:1030300015C08091730282FB222720F991E092272C
:1030400090FB82F990FB83F92CC080917402982F39
:10305000909591708E7F892B90FB81F980937402FB
:1030600022C00E944E088091730287FB222720F91C
:1030700091E0922790FB87F914C081E00E94480FED
:1030800012C08091730284FB222720F991E09227DD
:1030900090FB84F906C080917302982F909590FB65
:1030A00080F98093730280917302909174020E9460
:1030B000C20E0E944E0880E001C081E0DF91CF91F6
:1030C00008958FE891E00197F1F700C0000008959E
:1030D0000C94DE02CF93DF93A6E9B1E0C4E9D1E01E
:1030E00021E030E071E0A839B70759F18D91E82F60
:1030F000E295EF70F0E041A18F70B90102C0660F58
:10310000771F8A95E2F7CB01962F9095942391A390
:1031100092A1892B82A38991E82FE295EF70F0E0CC
:1031200041A18F70B90102C0660F771F8A95E2F73F
:10313000CB01962F9095942391A392A1892B82A3E2
:10314000D1CF0E94611883B182FB882780F94C9906
:1031500002C090E001C092E0892B8093340289B1D3
:10316000982F9170499902C080E001C082E0892BBC
:1031700080933502DF91CF9108954F925F926F92C5
:103180007F928F929F92AF92BF92CF92DF92EF92F7
:10319000FF920F931F93CF93DF9304E312E086E92E
:1031A000C82E81E0D82E94E9E92E91E0F92E22E391
:1031B000822E22E0922EC0E3D2E05801512C412C05
:1031C00034E0632E712CD501ED915D014E2F440F3B
:1031D000440FF60121916F01E22FE295EF70F0E0CC
:1031E00080A190E02F7002C0959587952A95E2F70F
:1031F00081709927D7015D917D01E52FE295EF70F0
:10320000F0E020A130E05F7002C0359527955A9517
:10321000E2F7F901E170FF2720FF02C0E2E0F0E0F1
:10322000E82BF92BE42BD801ED938D01EF70F0E042
:10323000EC57FE4F9081F4018081890F80838430A8
:103240004CF088818F5F888360E0852D0E9468182C
:1032500021E001C020E0D4018C918D3F44F48881AD
:103260008150888361E0852D0E94681821E0F40177
:103270008081082E000C990BB3010E945B27D401BA
:103280008D934D01422A53942196B2E05B129BCF5D
:10329000842DDF91CF911F910F91FF90EF90DF90E0
:1032A000CF90BF90AF909F908F907F906F905F90E6
:1032B0004F900895CF93DF9386319C4541F5EB0104
:1032C0000E94A10D982F8A81209102013091030163
:1032D000882379F09A7A81E009F480E080933602BD
:1032E000911102C069E201C065E3C9010E94C21EDA
:1032F0000AC080913602811102C069E201C065E313
:10330000C9010E94C41E0E94E30D80E001C081E05B
:10331000DF91CF9108958F929F92AF92BF92CF92FB
:10332000DF92EF92FF920F931F93CF93DF937C0175
:10333000DC01ED91FC91CF01815095458F3F9105C6
:1033400010F4B5E5FB27DB011296CC91CC2309F4F0
:10335000B4C2EF3FF10579F070F0EB32FD4519F0A2
:103360001092370260C39091370281E089278093E1
:103370003702A0E059C3A0913702AA2309F4EBC099
:1033800010923702E03CF10540F4E038F10508F016
:1033900073C0E034F105D0F505C0EF3FF10509F049
:1033A00008F4A0C021E030E040E050E060E070E0D0
:1033B00080E090E00E2F0E947527B09138022B2BF1
:1033C000B09139023B2BB0913A024B2BB0913B02AA
:1033D0005B2BB0913C026B2BB0913D027B2BB091EB
:1033E0003E028B2BB0913F029B2B209338023093EF
:1033F000390240933A0250933B0260933C0270932F
:103400003D0280933E0290933F02A1C021E030E054
:1034100040E050E060E070E080E090E08F01005418
:1034200011090E947527B09140022B2BB0914102E7
:103430003B2BB09142024B2BB09143025B2BB091DE
:1034400044026B2BB09145027B2BB09146028B2B33
:10345000B09147029B2B209340023093410240934E
:10346000420250934302609344027093450280935A
:103470004602909347026BC021E030E040E050E00C
:1034800060E070E080E090E08F01005811090E9438
:103490007527B09148022B2BB09149023B2BB0917C
:1034A0004A024B2BB0914B025B2BB0914C026B2B21
:1034B000B0914D027B2BB0914E028B2BB0914F02FD
:1034C0009B2B209348023093490240934A02509329
:1034D0004B0260934C0270934D0280934E02909386
:1034E0004F0235C021E030E040E050E060E070E0A5
:1034F00080E090E08F01005C11090E947527B09177
:1035000050022B2BB09151023B2BB09152024B2B0E
:10351000B09153025B2BB09154026B2BB0915502CA
:103520007B2BB09156028B2BB09157029B2B209393
:1035300050023093510240935202509353026093D1
:103540005402709355028093560290935702E701FC
:10355000F983E88369C2E034F105D0F4A090380221
:10356000B0903902C0903A02D0903B02E0903C0209
:10357000F0903D02B0913E0210913F0221E030E018
:1035800040E050E060E070E080E090E00E2F5DC031
:10359000E038F105E8F4A0904002B0904102C090FC
:1035A0004202D0904302E0904402F0904502B09174
:1035B00046021091470221E030E040E050E060E038
:1035C00070E080E090E04F01D0E48D1A91083CC09B
:1035D000E03CF105E8F4A0904802B0904902C090A8
:1035E0004A02D0904B02E0904C02F0904D02B09114
:1035F0004E0210914F0221E030E040E050E060E0E8
:1036000070E080E090E04F01D0E88D1A91081CC076
:10361000A0905002B0905102C0905202D09053023C
:10362000E0905402F0905502B0915602109157026A
:1036300021E030E040E050E060E070E080E090E0C9
:103640004F01D0EC8D1A9108082D0E947527A222F7
:10365000B322C422D522E622F722B823192321E07F
:1036600030E040E050E060E070E080E090E0E03486
:10367000F105A0F04F01E038F10520F4D0E48D1AF7
:1036800091080AC0E03CF10520F4D0E88D1A9108B9
:1036900003C0D0EC8D1A9108082D01C00E2F0E9496
:1036A00075270B2F0E948E2709F0BDC1E03CF10564
:1036B00048F4E038F10508F084C0E034F10508F082
:1036C00042C005C0EF3FF10509F008F4B8C021E0A1
:1036D00030E040E050E060E070E080E090E00E2FED
:1036E0000E9475272095309540955095609570956E
:1036F00080959095E09138022E23E09139023E2387
:10370000E0913A024E23E0913B025E23E0913C02BD
:103710006E23E0913D027E23E0913E028E23E091F4
:103720003F029E23209338023093390240933A029D
:1037300050933B0260933C0270933D0280933E02A3
:1037400090933F0271C18F010054110921E030E0D4
:1037500040E050E060E070E080E090E00E9475277B
:1037600020953095409550956095709580959095F1
:10377000E09140022E23E09141023E23E09142027B
:103780004E23E09143025E23E09144026E23E091D8
:1037900045027E23E09146028E23E09147029E235C
:1037A00020934002309341024093420250934302DF
:1037B00060934402709345028093460290934702BF
:1037C00033C18F010058110921E030E040E050E0A2
:1037D00060E070E080E090E00E94752720953095D1
:1037E000409550956095709580959095E091480230
:1037F0002E23E09149023E23E0914A024E23E091BC
:103800004B025E23E0914C026E23E0914D027E2339
:10381000E0914E028E23E0914F029E2320934802B6
:103820003093490240934A0250934B0260934C02FA
:1038300070934D0280934E0290934F02F5C08F011A
:10384000005C110921E030E040E050E060E070E011
:1038500080E090E00E947527209530954095509526
:103860006095709580959095E09150022E23E0919F
:1038700051023E23E09152024E23E09153025E2317
:10388000E09154026E23E09155027E23E0915602AE
:103890008E23E09157029E232093500230935102D1
:1038A0004093520250935302609354027093550216
:1038B0008093560290935702B7C0EF3FF10511F085
:1038C00008F0AEC0E034F105D0F4C0903802D090DA
:1038D0003902E0903A02F0903B0210913C02C09114
:1038E0003D02B0913E02A0913F0221E030E040E075
:1038F00050E060E070E080E090E00E2F5DC0E038C6
:10390000F105E8F4C0904002D0904102E0904202FC
:10391000F090430210914402C0914502B0914602DA
:10392000A091470221E030E040E050E060E070E02C
:1039300080E090E05F01D0E4AD1AB1083CC0E03C0B
:10394000F105E8F4C0904802D0904902E0904A02A4
:10395000F0904B0210914C02C0914D02B0914E027A
:10396000A0914F0221E030E040E050E060E070E0E4
:1039700080E090E05F01D0E8AD1AB1081CC0C090B3
:103980005002D0905102E0905202F09053021091F8
:103990005402C0915502B0915602A091570221E005
:1039A00030E040E050E060E070E080E090E05F01F7
:1039B000D0ECAD1AB1080A2D0E947527A22EAC20BA
:1039C000B32EBD20C42ECE20D52EDF20E62EE12240
:1039D000F72EFC22B823192F1A23E034F10570F0DA
:1039E000E038F10518F4E054F10908C0E03CF105B5
:1039F00018F4E058F10902C0E05CF10921E030E080
:103A000040E050E060E070E080E090E00E2F0E9427
:103A10007527A1E00B2F0E948E2719F4A0E001C0AA
:103A2000A1E0A17001C0AC2F8A2FDF91CF911F912F
:103A30000F91FF90EF90DF90CF90BF90AF909F904D
:103A40008F9008950F931F93CF93DF93C42FD22F9E
:103A5000FC0182818823C9F040935A020E94681FAA
:103A6000909359028093580280E28C0F883008F0BE
:103A700057C0C77081E001C0880FCA95EAF7DF918F
:103A8000CF911F910F910C94AB0580915A0248136E
:103A900030C080915802909159020E94801F883C4A
:103AA000910538F510E21D0FCD17B9F080E28C0FAB
:103AB000883040F4C77081E001C0880FCA95EAF7EA
:103AC0000E94B205183028F581E09D2F977001C043
:103AD000880F9A95EAF70E94AB05802F0E94A205F5
:103AE0001830F0F4D77081E001C0880FDA95EAF75A
:103AF0000AC080E28C0F883098F4C77081E001C062
:103B0000880FCA95EAF7DF91CF911F910F910C941E
:103B1000B205802FDF91CF911F910F910C94A205D8
:103B2000DF91CF911F910F9108950F939C01CB01CD
:103B3000243F4CE5340731F188F4293DFCE53F078B
:103B4000D9F02A3D4CE5340779F1283D3C45A9F5EB
:103B500006E221EE41EE68ED7CE52BC0263FFCE558
:103B60003F07E1F0A8F0273F3C4539F507E225EE95
:103B700046EE67EF7CE51DC007E225EE45EE69EDF8
:103B80007CE517C006E221EE40EE64EF7CE511C053
:103B900007E225EE44EE65EF7CE50BC006E221EE80
:103BA00042EE66EF7CE505C008E221E045EE6AEDF5
:103BB0007CE50E94221D80E008C0FC0182818823F0
:103BC00019F010925A0201C081E00F91089590936C
:103BD000A9018093A80108959093600280935F02E9
:103BE0000895E0915F02F0916002309721F001901A
:103BF000F081E02D099480E00895EF92FF920F93F9
:103C00001F93CF93DF93E0915F02F09160023097B2
:103C1000B1F18C010280F381E02D099580911F02A2
:103C200082FF2DC080FF04C082EE91E00E94ED0172
:103C3000E80118E08CEDE82E81E0F82E80911F025B
:103C400080FF0BC088811F928F93FF92EF920E949A
:103C500086020F900F900F900F9011502196111126
:103C6000EDCF80911F0280FF0AC08AED91E0DF91C5
:103C7000CF911F910F91FF90EF900C94ED01DF9188
:103C8000CF911F910F91FF90EF900895E0915F0207
:103C9000F0916002309739F022E0DC012C9304802F
:103CA000F581E02D0994089520915D0230915E0226
:103CB0002817390771F090935E0280935D02E091BE
:103CC0005F02F0916002309721F00680F781E02DCD
:103CD0000994089520915B0230915C0228173907FE
:103CE00071F090935C0280935B02E0915F02F0912F
:103CF0006002309721F00084F185E02D0994089549
:103D0000FC01329697E080E0915029F02191222326
:103D1000D9F38F5FF9CF0895662349F0FC013296FD
:103D200008962191621729F0E817F907D1F780E08A
:103D3000089581E008959C01FC0132969FEF80E098
:103D40004191461789F09F3F19F4411101C0982F06
:103D50008F5F8630A9F79F3F39F0F901E90FF11D18
:103D600097FDFA956283089508959C012A5F3F4F5D
:103D7000FC014281461301C012820196821793070B
:103D8000B9F708950C949B1E0C94B51E029626E07C
:103D9000FC0111922A95E9F7089508950C94CD1E1F
:103DA00083E0809361020C94CE1E811102C081E0F9
:103DB00001C082E0809361020C94CE1E0C94D51E4B
:103DC00081E0809361020C94CE1E0C94E01E089555
:103DD0000C94E71E0C94E81E0C94E71E0C94E71E4E
:103DE0000C94E71ECF930E94EE1E0E947C130E944B
:103DF000EC1EC0E08C2F0E947112811104C0CF5FB5
:103E0000C430C1F701C081E0CF91089508951F9299
:103E10000F920FB60F9211248F939F93AF93BF937E
:103E200080916202811113C080917D0290917E0287
:103E3000A0917F02B09180024196A11DB11D809397
:103E40007D0290937E02A0937F02B0938002BF9187
:103E5000AF919F918F910F900FBE0F901F9018956B
:103E600080918502843031F10E94FF03109262023A
:103E700020E488E190E00FB6F894A8958093600064
:103E80000FBE2093600083B7817F846083BF83B7B8
:103E9000816083BF7894889583B78E7F83BF0FB688
:103EA000F894A895809160008861809360001092DA
:103EB00060000FBE08950E944E080C94030482E037
:103EC00084BD93E095BD9AEF97BD80936E000895F1
:103ED0002FB7F89480917D0290917E02A0917F028D
:103EE000B09180022FBF08952FB7F89460917D02A2
:103EF00070917E0280917F02909180022FBF089581
:103F00009C014FB7F89480917D0290917E02A09120
:103F10007F02B09180024FBF821B930B089578946B
:103F20001F920F920FB60F9211248F939F93AF930E
:103F3000BF9380917D0290917E02A0917F02B0910B
:103F400080020196A11DB11D80937D0290937E0297
:103F5000A0937F02B0938002BF91AF919F918F9108
:103F60000F900FBE0F901F90189587E797E79093DB
:103F70000108809300089AE088E10FB6F894A895AC
:103F8000809360000FBE90936000FFCF809171021C
:103F90000895089522E02093E9002FEF3091E80082
:103FA000215035FD06C035ED3A95F1F7000021119D
:103FB000F5CF2091E80025FF0BC040E050E066E01F
:103FC00070E00E94B2228091E8008E778093E80032
:103FD0000895CF93DF9321E02093E9002FEF3091F4
:103FE000E800215035FD06C035ED3A95F1F70000A7
:103FF0002111F5CF2091E80025FF14C0EC0140E02D
:1040000050E068E070E00E94B2228091E8008E7774
:104010008093E80088E0FE01A9E6B2E001900D92ED
:104020008A95E1F7DF91CF910895809365027093AF
:1040300067026093660280918502843001F582E018
:104040008093E9008FEF9091E800815095FD06C0C4
:1040500095ED9A95F1F700008111F5CF8091E80078
:1040600085FF0DC040E050E063E070E085E692E03F
:104070000E94B2228091E8008E778093E800089534
:10408000BC0184E00C941520BC0183E00C94152045
:1040900088E092E00E94ED0180918402811109C0C4
:1040A0000E9443240E94A0248091E20084608093B7
:1040B000E200089584E092E00E94ED0110928402F3
:1040C000089580E092E00E94ED010C94E51E8CEFD3
:1040D00091E00E94ED016091810281E0611101C0D7
:1040E00080E00C94D01E88EF91E00E94ED01909149
:1040F000850281E0943009F080E0609181020C94A7
:10410000D51E209164022F5F822F62E30E944F2709
:10411000992319F02093640208951092640280910B
:104120006802882371F180918502843041F5809185
:10413000E9008F702091EC00922F917020FD90E8A3
:10414000892B93E09093E9009091EB0090FF14C0CD
:104150009091EE0097FF10C09091E80095FF03C08A
:104160001092F100F9CF9091E80090FF05C0909176
:10417000E8009E779093E8008F708093E90010929A
:104180006802089542E061EC81E00E94BC2342E2B3
:1041900061EC82E00E94BC2342E261EC83E00E9479
:1041A000BC239091850281E0943009F080E0609119
:1041B00081020C94DE1E80918702833009F461C075
:1041C00030F4813071F0823009F49AC008958A3059
:1041D00009F486C08B3009F46CC0893009F0A8C09E
:1041E00020C080918602813A09F0A2C08091E80047
:1041F000877F8093E80080918A0290918B02892BBF
:1042000021F468E089E692E003C060E080E090E09D
:1042100070E00E94FD228091E8008B778093E80097
:10422000089580918602813209F082C080918A02CD
:1042300090918B02029708F07BC08091E800877F05
:104240008093E8008091E80082FD05C0809185029E
:104250008111F8CF6DC02091F3008091F20090E0C1
:10426000922B029731F48091F100813011F0863069
:1042700021F48091F100809371028091E8008B77A6
:1042800053C080918602813A09F052C080918A021F
:1042900090918B02892B09F04BC08091E800877FB9
:1042A0008093E8008091E80080FFFCCF80911801A6
:1042B00036C0809186028132D9F580918A02909130
:1042C0008B02892BA9F58091E800877F8093E80015
:1042D0000E94F12380918802809318010C944E086B
:1042E00080918602813221F58091E800877F80935A
:1042F000E8000E94F1238091890280937202089560
:1043000080918602813AA1F48091E800877F8093B2
:10431000E8008091E80080FFFCCF809172028093DA
:10432000F1008091E8008E778093E8000C94F123EF
:1043300008959FB7F894109268029FBF90918502EC
:10434000943009F057C09091E9009F703091EC00D3
:10435000232F217030FD20E8922B23E02093E900E9
:104360002091EB0020FF43C02091EE0027FF3FC0CB
:1043700020916302222321F02091E80025FF37C01D
:104380001092630226E03091E80035FD15C03091AF
:104390008502343061F53091EB0035FD28C02150A5
:1043A00021F481E08093630222C0EFE9FFE03197BE
:1043B000F1F700C00000E7CF8093F1008091E800A2
:1043C00085FD0AC08091E80080FFFCCF8091E80065
:1043D0008E778093E80006C08FB7F89421E0209391
:1043E00068028FBF9F709093E90080E008959F70EE
:1043F0009093E9008FEF089584B7877F84BF0FB64D
:10440000F894A89580916000886180936000109274
:1044100060000FBE90E080E80FB6F89480936100D2
:10442000909361000FBE0C94E01E0E9443240E94F2
:10443000A024E2EEF0E080818460808378940C9484
:1044400034278CE091E00C94EC1D8091850285303E
:10445000C9F484EF91E00E94ED01809185028530DE
:1044600079F40E94301F809183028823B1F30E9467
:10447000F21E882391F30E949C220E944E08EDCFE9
:104480000C945B1F089508950C944622292F33271E
:1044900023303105C9F060F42130310581F022303C
:1044A000310509F041C08BE590E02AE332E040C0DD
:1044B00021323105E1F02232310531F135C082E19E
:1044C00090E025E932E034C099278130910549F028
:1044D00028F0029749F5ECE0F2E005C0E6E3F2E0EF
:1044E00002C0EEE1F2E0849190E09F0121C06330D0
:1044F0007105D0F4660F771FFB01EF55FE4F208149
:10450000318189E090E014C06330710568F4FB01EB
:10451000EE0FFF1FE556FE4F20813181FB01E8566B
:10452000FE4F808190E004C080E090E020E030E029
:10453000FA0131832083089580E189BD82E189BD3C
:1045400009B400FEFDCF8091D8008F7D8093D80004
:104550008091E00082608093E0008091E00081FD26
:10456000FCCF0895CF92DF92EF92FF920F931F93AB
:10457000CF93DF93EC018B017A010E94102481110B
:1045800033C0E114F10439F0F70180819181081BF7
:10459000190BC80FD91FC12CD12C0115110519F108
:1045A0008091E80085FD16C08091E8008E778093A9
:1045B000E800E114F10449F0F70180819181C80E0F
:1045C000D91ED182C08285E00FC00E9410248823AA
:1045D00021F30AC089918093F10001501109FFEF86
:1045E000CF1ADF0ADACF80E0DF91CF911F910F91D0
:1045F000FF90EF90DF90CF90089520918C02309142
:104600008D022617370748F06115710539F420919E
:10461000E8002E772093E80001C0B901FC0120E0FA
:104620006115710579F1809185028823F1F185305A
:10463000F1F18091E80083FD3CC08091E80082FDAB
:104640002EC08091E80080FFEBCF2091F300809195
:10465000F20090E0922B6115710551F088309105C0
:1046600038F421912093F100615071090196F3CF44
:1046700021E0089709F020E08091E8008E77809390
:10468000E800CECF2111CFCF0AC0809185028823C8
:1046900061F0853061F08091E80083FD0AC080916F
:1046A000E80082FFF2CF80E0089582E0089583E081
:1046B000089581E0089520918C0230918D02261793
:1046C000370748F06115710539F42091E8002E771D
:1046D0002093E80001C0B901FC0120E061157105DB
:1046E00091F180918502882309F440C0853009F456
:1046F0003FC08091E80083FD3DC08091E80082FDCD
:104700002FC08091E80080FFE9CF2091F3008091D5
:10471000F20090E0922B6115710559F088309105F7
:1047200040F424912093F100319661507109019673
:10473000F2CF21E0089709F020E08091E8008E7721
:104740008093E800CBCF2111CCCF0AC080918502A5
:10475000882361F0853061F08091E80083FD0AC014
:104760008091E80082FFF2CF80E0089582E0089512
:1047700083E0089581E00895982F973068F590932D
:10478000E900981739F07091EC002091ED005091FC
:10479000F00003C0242F762F50E021FD02C09F5F60
:1047A000ECCF3091EB003E7F3093EB003091ED0089
:1047B0003D7F3093ED003091EB0031603093EB00A2
:1047C0007093EC002093ED005093F0002091EE00E8
:1047D00027FDE5CF80E008958F708093E90081E0A8
:1047E00008958091860287FF11C08091E80082FDC4
:1047F00005C0809185028111F8CF11C08091E80039
:104800008B770BC080918502882349F08091E80066
:1048100080FFF8CF8091E8008E778093E8000895BC
:104820002091E4003091E50095E64091EC00842F62
:10483000817040FF23C08091E80080FD1DC0809101
:104840008502882399F0853099F08091EB0085FDF1
:1048500011C04091E4005091E5002417350729F379
:10486000915011F09A01E1CF84E0089582E008951B
:1048700083E0089581E0089580E008954091E80084
:1048800042FFDDCF08950E94B1240E94B924E0EEDA
:10489000F0E0808181608083E8EDF0E080818F77B7
:1048A000808319BCA7EDB0E08C918E7F8C938081C2
:1048B0008F7E80831092840208950F931F93CF936D
:1048C000DF930E94B1240E94B924C8EDD0E0888112
:1048D0008F77888388818068888388818F7D8883AB
:1048E00019BC1092850210928102109283021092DC
:1048F000820200EE10E0F80180818B7F8083888146
:104900008160888342E060E080E00E94BC23E1EEA9
:10491000F0E080818E7F8083E2EEF0E08081816034
:104920008083808188608083F80180818E7F80838E
:10493000888180618883DF91CF911F910F910895C5
:10494000E8EDF0E080818F7E8083E7EDF0E080810C
:104950008160808384E082BF81E0809384020C9434
:104960005D24E8EDF0E080818E7F80831092E2008C
:1049700008951092DA001092E10008951F920F92AC
:104980000FB60F9211242F933F934F935F936F9322
:104990007F938F939F93AF93BF93EF93FF938091F8
:1049A000E10082FF0BC08091E20082FF07C080918E
:1049B000E1008B7F8093E1000E9481208091DA00EA
:1049C00080FF1FC08091D80080FF1BC08091DA005B
:1049D0008E7F8093DA008091D90080FF0DC080E146
:1049E00089BD82E189BD09B400FEFDCF81E08093DD
:1049F00085020E94482005C019BC109285020E94C1
:104A00005A208091E10080FF19C08091E20080FF70
:104A100015C08091E2008E7F8093E2008091E200D9
:104A200080618093E2008091D80080628093D800FA
:104A300019BC85E0809385020E9467208091E10087
:104A400084FF30C08091E20084FF2CC080E189BDEA
:104A500082E189BD09B400FEFDCF8091D8008F7D31
:104A60008093D8008091E1008F7E8093E100809157
:104A7000E2008F7E8093E2008091E200816080936B
:104A8000E20080918102882311F084E007C08091C8
:104A9000E30087FD02C081E001C083E080938502CE
:104AA0000E9473208091E10083FF29C08091E20081
:104AB00083FF25C08091E100877F8093E10082E041
:104AC00080938502109281028091E1008E7F809315
:104AD000E1008091E2008E7F8093E2008091E2000D
:104AE00080618093E20042E060E080E00E94BC23AD
:104AF0008091F00088608093F0000E946120FF9117
:104B0000EF91BF91AF919F918F917F916F915F9145
:104B10004F913F912F910F900FBE0F901F901895BE
:104B20001F920F920FB60F9211242F933F934F9322
:104B30005F936F937F938F939F93AF93BF93CF9325
:104B4000DF93EF93FF93C091E900CF708091EC0069
:104B5000D82FD17080FDD0E81092E9008091F0004C
:104B6000877F8093F00078940E94D4251092E9000A
:104B70008091F00088608093F000CD2BCF70C093BF
:104B8000E900FF91EF91DF91CF91BF91AF919F919C
:104B90008F917F916F915F914F913F912F910F90E6
:104BA0000FBE0F901F9018951F93CF93DF93CDB733
:104BB000DEB7AA970FB6F894DEBF0FBECDBFE6E80A
:104BC000F2E08091F100819322E0EE38F207C9F71C
:104BD0000E94DB208091E80083FF2EC18091860235
:104BE00090918702492F50E04A30510508F024C1C6
:104BF000FA01EE59FF4F0C946F27803821F082386C
:104C000009F01AC108C08091820290918302992311
:104C100089F082600FC080918A028F70873008F01F
:104C20000BC18093E9008091EB0085FB882780F918
:104C30001092E9009091E800977F9093E8008093AC
:104C4000F1001092F100D1C0282F2D7F09F0F4C09F
:104C5000882319F0823061F0EFC0809188028130A2
:104C600009F0EAC0933009F080E0809383022EC0FF
:104C70008091880281112AC080918A028F702FEF63
:104C8000280F263008F0D8C08093E9002091EB006F
:104C900020FF1CC0933021F48091EB00806214C08F
:104CA0009091EB0090619093EB0021E030E0A9013E
:104CB00002C0440F551F8A95E2F74093EA00109214
:104CC000EA008091EB0088608093EB001092E9008D
:104CD0008091E800877F8093E8000E94F123ACC0B8
:104CE0008111AAC0109188021F778091E30080781B
:104CF000812B8093E3008091E800877F8093E80018
:104D00000E94F1238091E80080FFFCCF8091E300B6
:104D100080688093E300111102C082E001C083E04B
:104D20008093850289C08058823008F085C08091C8
:104D30008802909189028C3D53E0950779F583E0D4
:104D40008A838AE289834FB7F894DE01139620E0C4
:104D50003EE051E2E32FF0E050935700E49120FF52
:104D600003C0E295EF703F5FEF708E2F90E0EA3066
:104D700010F0C79601C0C0968D939D932F5F24318C
:104D800049F74FBF8091E800877F8093E8006AE28F
:104D900070E0CE0101960E94FD2216C060918A0249
:104DA00070918B02AE014F5F5F4F0E944422BC01A5
:104DB000892B09F441C09091E800977F9093E80017
:104DC00089819A810E945B238091E8008B77809390
:104DD000E80032C0803881F58091E800877F8093B9
:104DE000E800809181028093F1008091E8008E7745
:104DF00072CF811121C080918802909189029927F8
:104E00000297D4F48091E800877F8093E800809136
:104E10008802809381020E94F12380918102811196
:104E200006C08091E30087FD02C081E001C084E0FC
:104E3000809385020E94C2208091E80083FF0AC00F
:104E40008091E800877F8093E8008091EB0080628A
:104E50008093EB00AA960FB6F894DEBF0FBECDBFCD
:104E6000DF91CF911F910895CF9380918502882380
:104E7000A1F0C091E900CF709091EC00892F817072
:104E800090FD80E8C82B1092E9008091E80083FD36
:104E90000E94D425CF70C093E900CF910895991B4B
:104EA00079E004C0991F961708F0961B881F7A9521
:104EB000C9F78095089597FB072E16F4009407D044
:104EC00077FD09D00E94972707FC05D03EF4909506
:104ED00081959F4F0895709561957F4F0895EE0FCE
:104EE000FF1F0590F491E02D09940F93083090F086
:104EF000982F872F762F652F542F432F322F22275D
:104F00000850F4CF220F331F441F551F661F771F11
:104F1000881F991F0A95B2F70F9108952A153B052E
:104F20004C055D056E057F05800791070895AA1B56
:104F3000BB1B51E107C0AA1FBB1FA617B70710F084
:104F4000A61BB70B881F991F5A95A9F780959095B6
:104F5000BC01CD010895FB01DC0104C08D910190DD
:104F6000801921F441505040C8F7881B990B0895CF
:104F7000F999FECF92BD81BDF89A992780B5089521
:104F8000A8E1B0E042E050E00C94EC27262FF9991C
:104F9000FECF92BD81BDF89A019700B4021639F098
:104FA0001FBA20BD0FB6F894FA9AF99A0FBE089569
:104FB0000396272F0E94C7270E94C627252F0E94ED
:104FC000C727242F0C94C7270196272F0E94C72795
:104FD0000C94C627DC01CB01FC01F999FECF06C079
:104FE000F2BDE1BDF89A319600B40D9241505040A7
:084FF000B8F70895F894FFCF13
:104FF800C8000502280850011E0A1401C61FE91F2F
:10500800CA1F44204020C91F01E200E900EA00B598
:1050180000B600B700CD008301CC008A019201944C
:10502800012102230224022502260227022A02B3B2
:1050380000B4006F007000818283E200E900EA009A
:10504800B500B600B700CD008301CC008A019201FB
:1050580094012102230224022502260227022A02A1
:10506800B300B4006F0070008182836697C6343540
:10507800F4F5F6F700FF0100010000FFFF00000152
:105088000001FF0094913290407B224403C902A79B
:08509800024C0265027E0200D9
:00000001FF
